:103400000C94341A0C94461A0C94461A0C94461ACE
:103410000C94461A0C94461A0C94461A0C94461AAC
:103420000C94461A0C94461A0C94461A0C94461A9C
:103430000C94461A0C94461A0C94461A0C94461A8C
:103440000C94461A0C94461A0C94461A0C94461A7C
:103450000C94461A0C94461A0C94461A0C94461A6C
:103460000C94461A0C94461A11241FBECFEFD4E0D8
:10347000DEBFCDBF23E0A0E0B1E001C01D92AD3DB5
:10348000B207E1F70E943D1E0C94EC1E0C94001A4A
:10349000E0E0F0E0099508951F93CF93DF93EC01EE
:1034A000162F0E94C91E612FCE0193950E94C91E3E
:1034B00012BC11BCDF91CF911F9108950F931F9300
:1034C000CF93DF93EC018B010E94D71EB801CE0190
:1034D00093950E94D71E12BC11BCDF91CF911F9112
:1034E0000F910895519A3C9A3B9A08958091D10387
:1034F0008F5F8093D10391E09093BC029091B502CD
:10350000911105C080FD02C0439A01C0439880918B
:10351000B502813009F4439A8091D1038A3078F062
:103520001092D1038091B502811105C08091DC0316
:103530008A3028F401C080E08F5F8093DC03089517
:10354000CF93DF931092BB0210920301C1E0D0E051
:10355000CE010E94BB1E9091BB02980F9093BB02BC
:10356000909103018927809303012196CB30D105E7
:1035700079F712BC11BCDF91CF910895CF93DF93FF
:103580001092BB0210920301C1E0D1E0CE010E9473
:10359000BB1E9091BB02980F9093BB0290910301C8
:1035A0008927809303012196CB3081E0D80771F7FA
:1035B00012BC11BCDF91CF910895CF93DF9310928D
:1035C000BB0210920301C1E0D0E0CE010E94BB1EFD
:1035D0006091BB02680F6093BB0290910301892741
:1035E000809303012196CB30D10579F78EE090E0EE
:1035F0000E94C91E609103018FE090E00E94C91EE5
:103600006091BB028EE091E00E94C91E60910301AF
:103610008FE091E00E94C91E12BC11BCDF91CF91D6
:103620000895909100018091CE03981790F48091B5
:10363000C00085FD06C0E0ECF0E0A895808185FF24
:10364000FCCFE92FF0E0EF55FD4F80818093C6005D
:1036500001C04498809100018F5F8093000108951C
:103660009091C6008091CD03811151C0A89B08C0E4
:103670008091BA02813009F047C01092BA0204C0AA
:103680008091BA0281110DC09A32D9F5A89A16BC60
:103690001092CC038AE28093CB0381E08093BA023C
:1036A0000895813071F58091CC038F5F8093CC03B6
:1036B0008D3810F01092BA02E82FF0E0E85FFD4F6D
:1036C00090832091CB03392F320F3093CB0383307B
:1036D00041F434E0390F30939E023D3810F01092DF
:1036E000BA0230919E0283130CC02093CB03921335
:1036F00008C08091BA02813021F48093CD031092EA
:10370000BA02A89A16BC08958111FBCFBDCF0895C7
:103710002091A40244E0420F85E0820F8093CE0303
:10372000442369F0E1EAF2E02D5F30E02E553D4F91
:1037300080E09191890FE217F307D9F701C080E08B
:10374000E42FF0E0EF55FD4F808381E0809300018E
:10375000449A86E69EE00197F1F700008091C00050
:1037600085FD06C0E0ECF0E0A895808185FFFCCFE8
:103770008091A1028093C6000895CF92DF92EF92CC
:10378000FF92CF93DF938091BD029091BE02A091F2
:10379000BF02B091C0028093D2039093D303A09351
:1037A000D403B093D5034091B6025091B702609113
:1037B000B8027091B90284179507A607B707C1F13F
:1037C000C090D603D090D703E090D803F090D903EF
:1037D000C4E0D1E0E1ECF2E040E050E09A01ABEA75
:1037E000BAEA0E94AC1E969587959C01220F331F62
:1037F000820F931F4817590721F08081841B8F5F28
:1038000004C080819EEF940F890FC80ED11CE11C6B
:10381000F11C89934F5F5F4F319640385105F1F6A7
:10382000C092D603D092D703E092D803F092D90386
:10383000DF91CF91FF90EF90DF90CF900895A89502
:1038400061E081E090E00E944C1A60E070E084E06A
:1038500090E00E945E1A60E070E086E090E00E94D6
:103860005E1A60E070E088E090E00E945E1A6EEF01
:103870008AE090E00E944C1AA8950E94DD1A0895F3
:1038800085E0A895439A2FEF3FE392E02150304026
:103890009040E1F700C0000043982FEF3FE392E033
:1038A000215030409040E1F700C00000815049F7BE
:1038B00008951F93CF93DF9381E090E00E94BB1E99
:1038C000813041F081E091E00E94BB1E813011F017
:1038D0000E941F1CA8958EE090E00E94BB1EC82F7E
:1038E0008FE090E00E94BB1ED82F0E94A01A80910A
:1038F000BB02C81307C0C1E0809103018D1719F006
:10390000C0E001C0C0E0A8958EE091E00E94BB1E1F
:10391000D82F8FE091E00E94BB1E182F0E94BE1A84
:103920008091BB02D81304C080910301181751F194
:10393000CC2389F12AC0A895C1E0D0E0A895CE019A
:1039400093950E94BB1E682FCE010E94C91E21962E
:10395000CB30D10599F70E94DD1A0E94401C2BC084
:10396000A895CE010E94BB1E682FCE0193950E94A0
:10397000C91E2196CB30D10599F70E94DD1A0E940D
:10398000401C19C0CC23B9F216C0C130A1F4A895CF
:10399000C1E0D0E0E5CF0E941F1C0E94401CA8950A
:1039A0002FEF8FE796E1215080409040E1F700C073
:1039B00000000E94401CDF91CF911F910895CF928B
:1039C000DF92EF92FF921F93CF93DF93C0910A0291
:1039D0008091A002C81349C1E8E0F2E01181D481CE
:1039E000D130A9F580910D02813039F58093B5026F
:1039F000E1EAF2E09AE29083C18312839CE0938330
:103A0000848385838FE090E09783868381E092E0D2
:103A1000918780878091CF039091D003938782878D
:103A20008091DA039091DB039587848780E890E0AA
:103A3000978786870E94881B18C11092B502823032
:103A400009F057C08EEF80930C0280E01BC0D2308B
:103A5000C1F48091B502813009F0A2C060910D02DD
:103A60008EEF860F8D3F08F09DC06093A0028AE024
:103A700090E00E944C1A0E94DD1A1092B50281E07B
:103A800001C080E090910C029330A1F59091B502B5
:103A9000913009F0B7C0E8E0F2E0668170E0762F7F
:103AA00066278581680F711D7093D0036093CF03E3
:103AB00088E090E00E945E1A6FEF83E090E00E9441
:103AC0004C1A0E94DD1A1092D6031092D70310925E
:103AD000D8031092D90380E090E0A0E0BFEF80937C
:103AE000B6029093B702A093B802B093B90281E0F6
:103AF00001C080E090910C02953009F056C0909181
:103B0000B502913009F0A3C080910D0290910E0290
:103B1000A0910F02B09110028093BD029093BE025B
:103B2000A093BF02B093C002E3E1F2E0A1ECB2E0E7
:103B300023E932E081918D932E173F07D9F70E9438
:103B4000BD1B6091D2037091D3038091D4039091F7
:103B5000D50361152AE172078105910528F5C0900A
:103B6000B602D090B702E090B802F090B9026C159E
:103B70007D058E059F0511F00E94841F8091D20360
:103B80009091D303A091D403B091D5038093B60252
:103B90009093B702A093B802B093B90281E005C038
:103BA00080E003C080E001C080E090910C02993079
:103BB00049F59091B502913009F049C0C0900D02CD
:103BC000D0900E02E0900F02F09010024091D603C8
:103BD0005091D7036091D8037091D90381E0C41646
:103BE000D506E606F70609F080E0C416D506E60617
:103BF000F70669F561E083E090E00E944C1A0E94AC
:103C0000DD1A81E090910C029E3F09F5E1EAF2E0B5
:103C10008AE28083C183128384E083838EEF84836E
:103C20008FE085838091CF039091D0039783868323
:103C300083E090E00E94BB1E813021F01092A80228
:103C40001092A70212BC11BC0E94881B0EC0E1EAB0
:103C5000F2E09AE29083C183128393E0938394E627
:103C60009483D58386830E94881BDF91CF911F9117
:103C7000FF90EF90DF90CF900895A895C8E18FE076
:103C80000FB6F894A895C09360000FBE80936000B3
:103C90000E94721A0E94591C84E090E00E94C31E88
:103CA0009093DB038093DA0386E090E00E94C31ECA
:103CB000909302018093010188E090E00E94C31E6E
:103CC0009093D0038093CF038AE090E00E94BB1EC4
:103CD0008093A00212BC11BC1092C5008FE28093A9
:103CE000C400C093C10084E085BD8BE08093810057
:103CF00080E09AE59093890080938800C0ECD0E042
:103D000018E0A895B19B03C0B19A0E94761A8881E9
:103D1000882314F40E94301B888186FF05C08881A7
:103D2000806488830E94111B8091CD03882321F039
:103D30000E94DF1C1092CD038091DC0384508430FC
:103D400000F71093DC0383E090E00E94BB1E8130FB
:103D5000C1F60E94481AD5CFA29FB001B39FC001FF
:103D6000A39F700D811D1124911DB29F700D811DA7
:103D70001124911D0895F999FECF92BD81BDF89A45
:103D8000992780B50895A8E1B0E042E050E00C9496
:103D9000DE1E262FF999FECF1FBA92BD81BD20BD30
:103DA0000FB6F894FA9AF99A0FBE019608950E94F8
:103DB000C91E272F0C94CA1EDC01CB01FC01F99906
:103DC000FECF06C0F2BDE1BDF89A319600B40D9267
:0C3DD00041505040B8F70895F894FFCF20
:103F0000E0E0FAE109950895CF92DF92EF92FF92F7
:103F1000CF93DF936B017C01A8956FB7F999FECF22
:103F2000A60183E0F60180935700E89507B600FCF0
:103F3000FDCFC4E8D1E0A4E0B1E031E0445051400D
:103F4000FA01EA0FFB1F11968C91119790E0982FC0
:103F500088272C91820F911D0C0130935700E89512
:103F600011241296AC17BD0759F785E0F60180932E
:103F70005700E89507B600FCFDCF81E1809357001C
:103F8000E8956FBFDF91CF91FF90EF90DF90CF90DA
:023F9000089592
:0400000300003400C5
:00000001FF
